:1000000028288F018E00FF308E07031C8F07031CEA
:10001000232803308D00DF300F2003288D01E83EB8
:100020008C008D09FC30031C18288C070318152838
:100030008C0764008D0F15280C181E288C1C222894
:1000400000002228080083130313831264000800B1
:100050008316FF30850086018312860105308F00EC
:10006000DC3002200130A6006400053026020318AF
:10007000822B64002608013C031D4228E830A400BE
:100080000330A50064002608023C031D4B28F43011
:10009000A4000130A50064002608033C031D53287A
:1000A000FA30A400A50164002608043C031D5B2867
:1000B0006430A400A50106148316061083122508D7
:1000C0008F002408022086148316861083122508C8
:1000D0008F002408022006158316061183122508B6
:1000E0008F002408022086158316861183122508A6
:1000F0008F00240802200616831606128312250894
:100100008F00240802208616831686128312250883
:100110008F00240802200617831606138312250871
:100120008F00240802208617831686138312250861
:100130008F0024080220061083160610831225085B
:100140008F0024080220861083168610831225084B
:100150008F00240802200611831606118312250839
:100160008F00240802208611831686118312250829
:100170008F00240802200612831606128312250817
:100180008F00240802208612831686128312250807
:100190008F002408022006138316061383122508F5
:1001A0008F002408022086138316861383120330DF
:1001B0008F00E830022006148316061083122508EB
:1001C0008F002408022086148316861083122508C7
:1001D0008F002408022006158316061183122508B5
:1001E0008F002408022086158316861183122508A5
:1001F0008F00240802200616831606128312250893
:100200008F00240802208616831686128312250882
:100210008F00240802200617831606138312250870
:100220008F00240802208617831686138312250860
:100230008F00240802208613831686138312250854
:100240008F00240802200613831606138312250844
:100250008F00240802208612831686128312250836
:100260008F00240802200612831606128312250826
:100270008F00240802208611831686118312250818
:100280008F00240802200611831606118312250808
:100290008F002408022086108316861083122508FA
:1002A0008F002408022006108316061083120330E4
:1002B0008F00E830022006148316061083122508EA
:1002C0008F002408022086148316861083120610DD
:1002D00083160610831225088F00240802200615B5
:1002E0008316061183128610831686108312250842
:1002F0008F002408022086158316861183120611AA
:1003000083160611831225088F0024080220061682
:10031000831606128312861183168611831225080E
:100320008F00240802208616831686128312061276
:1003300083160612831225088F0024080220061750
:1003400083160613831286128316861283122508DB
:100350008F00240802208617831686138312061343
:1003600083160613831225088F00240802208613A3
:1003700083168613831225088F0024080220033079
:100380008F00E83002208617831686138312250813
:100390008F00240802200617831606138312861383
:1003A00083168613831225088F00240802208616E0
:1003B00083168612831206138316061383122508EA
:1003C0008F00240802200616831606128312861256
:1003D00083168612831225088F00240802208615B2
:1003E00083168611831206128316061283122508BD
:1003F0008F00240802200615831606118312861129
:1004000083168611831225088F0024080220861483
:10041000831686108312061183160611831225088F
:100420008F002408022006148316061083128610FB
:1004300083168610831225088F00240802200610D8
:1004400083160610831225088F002408022003302B
:100450008F00E8300220FF30860025088F00240836
:100460000220061083160610831225088F00240828
:100470000220061483160610831286108316861037
:10048000831225088F002408022086148316861004
:100490008312061183160611831225088F00240883
:1004A0000220061583160611831286118316861103
:1004B000831225088F0024080220861583168611D2
:1004C0008312061283160612831225088F00240851
:1004D00002200616831606128312861283168612CF
:1004E000831225088F0024080220861683168612A0
:1004F0008312061383160613831225088F0024081F
:10050000022006178316061383128613831686139A
:10051000831225088F00240802208617831686136D
:10052000831203308F00E8300220FF308600250858
:100530008F00240802208613831686138312250851
:100540008F002408022006138316061383128617D1
:1005500083168613831225088F0024080220861232
:100560008316861283120617831606138312250834
:100570008F002408022006128316061283128616A4
:1005800083168612831225088F0024080220861104
:100590008316861183120616831606128312250807
:1005A0008F002408022086158316861183120611F7
:1005B00083160611831225088F00240802200615D1
:1005C000831606118312861083168610831225085F
:1005D0008F002408022086148316861083120610CA
:1005E00083160610831225088F00240802200614A3
:1005F00083160610831203308F00E8300220860134
:1006000001308F002C30022006148316061083124E
:10061000861783168613831225088F00240802206C
:100620008614831686108312061783160613831208
:1006300025088F0024080220061583160611831250
:10064000861683168612831225088F00240802203E
:1006500086158316861183120616831606128312D8
:1006600025088F0024080220861183168611831224
:10067000061283160612831225088F002408022012
:1006800086128316861283120611831606118312B0
:1006900025088F00240802200613831606138312F0
:1006A000861083168610831225088F0024080220E6
:1006B0008613831686138312061083160610831280
:1006C00025088F002408022003308F00E830022024
:1006D0000130A70064000330270203187C2BFF3091
:1006E000860001308F002C300220860101308F00FF
:1006F0002C300220A70F6A2B03308F00E830022035
:10070000A60F342803308F00E83002200130A60005
:100710006400043026020318962BFF308600C83090
:1007200001208601C8300120A60F882B03308F00DE
:0A073000E8300220322863009B2B02
:02400E00F53F7C
:00000001FF
